:020000040800F2
:10000000B0090020010100080D3D00083D3B00083B
:10001000093D00083D1D00084D410008000000009A
:10002000000000000000000000000000294000085F
:10003000AD1D000800000000113D00082D40000823
:100040001B0100081B0100081B0100081B01000820
:100050001B0100081B0100081B0100081B01000810
:100060001B0100081B0100081B0100081B01000800
:100070001B0100081B0100081B0100081B010008F0
:100080001B0100081B0100081B0100081B010008E0
:100090001B0100081B0100081B0100081B010008D0
:1000A0001B0100081B0100081B0100081B010008C0
:1000B0001B0100081B0100081B0100081B010008B0
:1000C0001B0100081B0100081B0100081B010008A0
:1000D0001B010008414100081B0100081B0100082A
:1000E0001B0100081B0100081B010008DFF80CD0F1
:1000F00000F014F900480047A9410008B0090020A9
:100100000648804706480047FEE7FEE7FEE7FEE7B1
:10011000FEE7FEE7FEE7FEE7FEE7FEE73140000808
:10012000ED000008F0B480EA0102D40F4200B2EB07
:10013000410F02D20246084611464A0042D0C30D82
:10014000DDB2C1F3C752AD1A202D35DAC1F3160165
:1001500041F4000204B15242C5F1200602FA06F150
:100160002A411044B3EBD05F23D0C4B1012DA0EBE2
:10017000C35009DCF0BC4FF0004202EAC352DBB2CC
:1001800000F5000000F09CB8400000F1807000EB2A
:10019000C350A0F1807040EAD170490009E04908DD
:1001A00041EAC071A0EBC35000F50000400800EB2D
:1001B000C350F0BC00F07BB86142012202EB410168
:1001C000001BF6E7F0BC704781F00041AAE780F021
:1001D0000040A7E780EA010210B502F000434000AA
:1001E00022D04A001FD0010E01EB1261C0F356006D
:1001F000C2F3560240F4000042F40002A0FB0220C9
:1002000000047F39140400D0401C50EA124001D48D
:100210004000491EC2B20C0604EBD010401C40083E
:10022000802A02D003E0002010BD20F00100002948
:1002300000DA0020184310BDC10F80EAE0700844C6
:10024000CA079623002100F03BB8962300221146EE
:1002500000F036B800F0004220F00040C10DC0F3BD
:10026000160040F400007F2901DA0020704796292B
:1002700003DCC1F19601C84001E096398840002AAC
:10028000F4D04042704720F00040C10DC0F316008A
:1002900040F400007F2901DA00207047962903DC32
:1002A000C1F19601C84070479639884070470029CF
:1002B000A8BF7047401C490008BF20F001007047EC
:1002C00010B4B0FA80FC00FA0CF050EA010404BF4C
:1002D00010BC704749B1CCF1200421FA04F411FAA2
:1002E0000CF118BF012121430843A3EB0C01CB1DE6
:1002F0004FEA00614FEA102042BF002010BC704757
:1003000000EBC35010440029A4BF10BC7047401C30
:10031000490008BF20F0010010BC7047064C074D93
:1003200006E0E06840F0010394E8070098471034C5
:10033000AC42F6D3FFF7DEFE186100083861000812
:1003400040F218000021C2F20000002283188154FC
:1003500002F58072B2F5806F19721974197683F8FC
:10036000201083F8281083F8301083F8381083F8B1
:10037000401083F8481083F8501083F8581083F821
:10038000601083F8681083F8701083F8781083F891
:10039000801083F8881083F8901083F8981083F801
:1003A000A01083F8A81083F8B01083F8B81083F871
:1003B000C01083F8C81083F8D01083F8D81083F8E1
:1003C000E01083F8E81083F8F01083F8F810BDD13E
:1003D00000210022831802F58072B2F5806F5970F7
:1003E00059725974597683F8211083F8291083F8CB
:1003F000311083F8391083F8411083F8491083F8DD
:10040000511083F8591083F8611083F8691083F84C
:10041000711083F8791083F8811083F8891083F8BC
:10042000911083F8991083F8A11083F8A91083F82C
:10043000B11083F8B91083F8C11083F8C91083F89C
:10044000D11083F8D91083F8E11083F8E91083F80C
:10045000F11083F8F910BDD100210022831802F5B4
:100460008072B2F5806F997099729974997683F859
:10047000221083F82A1083F8321083F83A1083F898
:10048000421083F84A1083F8521083F85A1083F808
:10049000621083F86A1083F8721083F87A1083F878
:1004A000821083F88A1083F8921083F89A1083F8E8
:1004B000A21083F8AA1083F8B21083F8BA1083F858
:1004C000C21083F8CA1083F8D21083F8DA1083F8C8
:1004D000E21083F8EA1083F8F21083F8FA10BDD125
:1004E00000210022831802F58072B2F5806FD97066
:1004F000D972D974D97683F8231083F82B1083F836
:10050000331083F83B1083F8431083F84B1083F8C3
:10051000531083F85B1083F8631083F86B1083F833
:10052000731083F87B1083F8831083F88B1083F8A3
:10053000931083F89B1083F8A31083F8AB1083F813
:10054000B31083F8BB1083F8C31083F8CB1083F883
:10055000D31083F8DB1083F8E31083F8EB1083F8F3
:10056000F31083F8FB10BDD100210022831802F59F
:100570008072B2F5806F197119731975197783F844
:10058000241083F82C1083F8341083F83C1083F87F
:10059000441083F84C1083F8541083F85C1083F8EF
:1005A000641083F86C1083F8741083F87C1083F85F
:1005B000841083F88C1083F8941083F89C1083F8CF
:1005C000A41083F8AC1083F8B41083F8BC1083F83F
:1005D000C41083F8CC1083F8D41083F8DC1083F8AF
:1005E000E41083F8EC1083F8F41083F8FC10BDD10C
:1005F00000210022831802F58072B2F5806F5971D4
:1006000059735975597783F8251083F82D1083F89D
:10061000351083F83D1083F8451083F84D1083F8AA
:10062000551083F85D1083F8651083F86D1083F81A
:10063000751083F87D1083F8851083F88D1083F88A
:10064000951083F89D1083F8A51083F8AD1083F8FA
:10065000B51083F8BD1083F8C51083F8CD1083F86A
:10066000D51083F8DD1083F8E51083F8ED1083F8DA
:10067000F51083F8FD10BDD100210022831802F58A
:100680008072B2F5806F997199739975997783F833
:10069000261083F82E1083F8361083F83E1083F866
:1006A000461083F84E1083F8561083F85E1083F8D6
:1006B000661083F86E1083F8761083F87E1083F846
:1006C000861083F88E1083F8961083F89E1083F8B6
:1006D000A61083F8AE1083F8B61083F8BE1083F826
:1006E000C61083F8CE1083F8D61083F8DE1083F896
:1006F000E61083F8EE1083F8F61083F8FE10BDD1F3
:1007000000210022831802F58072B2F5806FD97142
:10071000D973D975D97783F8271083F82F1083F808
:10072000371083F83F1083F8471083F84F1083F891
:10073000571083F85F1083F8671083F86F1083F801
:10074000771083F87F1083F8871083F88F1083F871
:10075000971083F89F1083F8A71083F8AF1083F8E1
:10076000B71083F8BF1083F8C71083F8CF1083F851
:10077000D71083F8DF1083F8E71083F8EF1083F8C1
:10078000F71083F8FF10BDD100F002BD2DE9F04F46
:1007900002FB02FCBCEB4C0F88BFBDE8F08F40F2BF
:1007A00018084FF0000B4FF0010EC2F2000800BF16
:1007B0000BEB00058E1AF7B2EDB2FF0808EBC5058A
:1007C00006F00706EC5D0EFA06F944EA0904EC555A
:1007D000A0EB0B04E4B208EBC404E65D46EA0906AC
:1007E000E6555618F7B2FF0806F0070914F807A0F7
:1007F0000EFA09F64AEA0603E355EB5D0BEB01043A
:100800003343EB551318E5B2DBB2ED0808EBC30335
:1008100004F007045E5D0EFA04F946EA09065E5527
:10082000A1EB0B06F7B2FF0806F00706DC5D0EFA37
:1008300006F63443DC55831ADBB208EBC303DC5DF8
:100840003443DC550BF1010602FB02F706FB067789
:100850005C5D67458CBF013AB34602FB02F644EA91
:100860000904BCEB460F5C55A2DDBDE8F08F00002B
:100870002DE9F04F82B0151AB2EB000A18BF4FF005
:10088000FF3A002D019544BF6A420192012DA3EB6E
:1008900001044FF00102A8BF92465B1A9946019AE3
:1008A0001CBFC2F100094FF0FF33002CC4BFA146AA
:1008B0000123CB4600934A45C8BF93460027002238
:1008C000002400BF40F218065FFA80FEC2F2000664
:1008D000C1F3C40806EBCE0E01F007031EF8086052
:1008E000012505FA03F3DDF82CC046EA0305BCF147
:1008F000000F08BF26EA0305019B07EB0906134416
:10090000B3EB0B02D4BF1A465044B6EB0B07D8BF6B
:100910003746009B04F10104C8BF1944A3B29B45AC
:100920000EF80850CED202B0BDE8F08FB0B5CD08B9
:1009300001F0070E40F21801C2F2000101EBC00005
:100940004FF0010C415D0CFA0EF341EA0304002A5A
:1009500008BF21EA03044455B0BD00002DE9F04171
:1009600082B040F60044C4F2010420464FF48041B6
:100970000022002601F032FF20464FF48041012280
:1009800001F02CFFAE208DF8070020464FF4805177
:10099000002201F023FF40F20855C2F200050DF1DC
:1009A0000701284601224FF47A7302F043FC4FF00E
:1009B000200820464FF4805100228DF8078001F076
:1009C0000DFF0DF10701284601224FF47A7302F062
:1009D00031FC102720464FF4805100228DF807701B
:1009E00001F0FCFE0DF10701284601224FF47A7355
:1009F00002F020FCB0208DF8070020464FF4805113
:100A0000002201F0EBFE0DF10701284601224FF410
:100A10007A7302F00FFCC8208DF8070020464FF4CF
:100A20008051002201F0DAFE0DF107012846012273
:100A30004FF47A7302F0FEFB20464FF480510022FF
:100A40008DF8076001F0CAFE0DF10701284601226A
:100A50004FF47A7302F0EEFB20464FF480510022EF
:100A60008DF8077001F0BAFE0DF10701284601224A
:100A70004FF47A7302F0DEFB40208DF80700204629
:100A80004FF48051002201F0A9FE0DF10701284624
:100A900001224FF47A7302F0CDFB81208DF807001C
:100AA00020464FF48051002201F098FE0DF107011D
:100AB000284601224FF47A7302F0BCFBFF208DF828
:100AC000070020464FF48051002201F087FE0DF10F
:100AD0000701284601224FF47A7302F0ABFBA120F4
:100AE0008DF8070020464FF48051002201F076FE79
:100AF0000DF10701284601224FF47A7302F09AFBA8
:100B0000A6208DF8070020464FF48051002201F006
:100B100065FE0DF10701284601224FF47A7302F0B9
:100B200089FBA8208DF8070020464FF48051002251
:100B300001F054FE0DF10701284601224FF47A73AB
:100B400002F078FB3F208DF8070020464FF48051DB
:100B5000002201F043FE0DF10701284601224FF467
:100B60007A7302F067FBA4208DF8070020464FF44B
:100B70008051002201F032FE0DF1070128460122CA
:100B80004FF47A7302F056FBD3208DF8070020460D
:100B90004FF48051002201F021FE0DF1070128469B
:100BA00001224FF47A7302F045FB20464FF4805146
:100BB00000228DF8076001F011FE0DF107012846B3
:100BC00001224FF47A7302F035FBD5208DF807002F
:100BD00020464FF48051002201F000FE0DF1070184
:100BE000284601224FF47A7302F024FBF0208DF89E
:100BF000070020464FF48051002201F0EFFD0DF177
:100C00000701284601224FF47A7302F013FBD92022
:100C10008DF8070020464FF48051002201F0DEFDE0
:100C20000DF10701284601224FF47A7302F002FB0E
:100C300022208DF8070020464FF48051002201F059
:100C4000CDFD0DF10701284601224FF47A7302F021
:100C5000F1FADA208DF8070020464FF48051002287
:100C600001F0BCFD0DF10701284601224FF47A7313
:100C700002F0E0FA12208DF8070020464FF4805170
:100C8000002201F0ABFD0DF10701284601224FF4CF
:100C90007A7302F0CFFADB208DF8070020464FF47C
:100CA0008051002201F09AFD0DF107012846012232
:100CB0004FF47A7302F0BEFA20464FF480510022BE
:100CC0008DF8078001F08AFD0DF107012846012209
:100CD0004FF47A7302F0AEFA8D208DF807002046AB
:100CE0004FF48051002201F079FD0DF107012846F3
:100CF00001224FF47A7302F09DFA14208DF8070058
:100D000020464FF48051002201F068FD0DF10701EB
:100D1000284601224FF47A7302F08CFAAF208DF846
:100D2000070020464FF48051002201F057FD0DF1DD
:100D30000701284601224FF47A7302F07BFA40F251
:100D40001800C2F2000000214218465401F58071DB
:100D5000B1F5806F16721674167682F8206082F8EC
:100D6000286082F8306082F8386082F8406082F84B
:100D7000486082F8506082F8586082F8606082F8BB
:100D8000686082F8706082F8786082F8806082F82B
:100D9000886082F8906082F8986082F8A06082F89B
:100DA000A86082F8B06082F8B86082F8C06082F80B
:100DB000C86082F8D06082F8D86082F8E06082F87B
:100DC000E86082F8F06082F8F860BDD1002100226E
:100DD000831802F58072B2F5806F59705972597498
:100DE000597683F8211083F8291083F8311083F89D
:100DF000391083F8411083F8491083F8511083F8B3
:100E0000591083F8611083F8691083F8711083F822
:100E1000791083F8811083F8891083F8911083F892
:100E2000991083F8A11083F8A91083F8B11083F802
:100E3000B91083F8C11083F8C91083F8D11083F872
:100E4000D91083F8E11083F8E91083F8F11083F8E2
:100E5000F910BDD100210022831802F58072B2F58D
:100E6000806F997099729974997683F8221083F83B
:100E70002A1083F8321083F83A1083F8421083F86E
:100E80004A1083F8521083F85A1083F8621083F8DE
:100E90006A1083F8721083F87A1083F8821083F84E
:100EA0008A1083F8921083F89A1083F8A21083F8BE
:100EB000AA1083F8B21083F8BA1083F8C21083F82E
:100EC000CA1083F8D21083F8DA1083F8E21083F89E
:100ED000EA1083F8F21083F8FA10BDD10021002245
:100EE000831802F58072B2F5806FD970D972D97407
:100EF000D97683F8231083F82B1083F8331083F806
:100F00003B1083F8431083F84B1083F8531083F899
:100F10005B1083F8631083F86B1083F8731083F809
:100F20007B1083F8831083F88B1083F8931083F879
:100F30009B1083F8A31083F8AB1083F8B31083F8E9
:100F4000BB1083F8C31083F8CB1083F8D31083F859
:100F5000DB1083F8E31083F8EB1083F8F31083F8C9
:100F6000FB10BDD100210022831802F58072B2F57A
:100F7000806F197119731975197783F8241083F824
:100F80002C1083F8341083F83C1083F8441083F855
:100F90004C1083F8541083F85C1083F8641083F8C5
:100FA0006C1083F8741083F87C1083F8841083F835
:100FB0008C1083F8941083F89C1083F8A41083F8A5
:100FC000AC1083F8B41083F8BC1083F8C41083F815
:100FD000CC1083F8D41083F8DC1083F8E41083F885
:100FE000EC1083F8F41083F8FC10BDD1002100222E
:100FF000831802F58072B2F5806F59715973597573
:10100000597783F8251083F82D1083F8351083F86D
:101010003D1083F8451083F84D1083F8551083F880
:101020005D1083F8651083F86D1083F8751083F8F0
:101030007D1083F8851083F88D1083F8951083F860
:101040009D1083F8A51083F8AD1083F8B51083F8D0
:10105000BD1083F8C51083F8CD1083F8D51083F840
:10106000DD1083F8E51083F8ED1083F8F51083F8B0
:10107000FD10BDD100210022831802F58072B2F567
:10108000806F997199739975997783F8261083F811
:101090002E1083F8361083F83E1083F8461083F83C
:1010A0004E1083F8561083F85E1083F8661083F8AC
:1010B0006E1083F8761083F87E1083F8861083F81C
:1010C0008E1083F8961083F89E1083F8A61083F88C
:1010D000AE1083F8B61083F8BE1083F8C61083F8FC
:1010E000CE1083F8D61083F8DE1083F8E61083F86C
:1010F000EE1083F8F61083F8FE10BDD10021002217
:10110000831802F58072B2F5806FD971D973D975E1
:10111000D97783F8271083F82F1083F8371083F8D6
:101120003F1083F8471083F84F1083F8571083F867
:101130005F1083F8671083F86F1083F8771083F8D7
:101140007F1083F8871083F88F1083F8971083F847
:101150009F1083F8A71083F8AF1083F8B71083F8B7
:10116000BF1083F8C71083F8CF1083F8D71083F827
:10117000DF1083F8E71083F8EF1083F8F71083F897
:10118000FF10BDD100F004F802B0BDE8F08100000E
:101190002DE9F04F81B040F6004440F2180640F2CD
:1011A0000855C4F20104C2F20006C2F200050DF1B6
:1011B00001090DF1020B0DF103074FF0000800BF0C
:1011C000A8F150008DF8000020464FF48051002215
:1011D00001F004FB2846694601224FF47A7302F0BD
:1011E00029F800208DF8010020464FF4805100229C
:1011F00001F0F4FA2846494601224FF47A7302F0CE
:1012000019F810208DF8020020464FF4805100227A
:1012100001F0E4FA2846594601224FF47A7302F0AD
:1012200009F86FF0070A00BF06EB0A00007A4FF4D6
:1012300080518DF803002046012201F0CFFA2846A4
:10124000394601224FF47A7301F0F4FF0AF1080ADB
:10125000BAF57E7FE8D108F10108B8F1080F06F170
:101260000106ADD101B0BDE8F08F00002DE9F04FCF
:1012700087B0082B049001D106250BE0D808012780
:101280005E0718BF07EBD3005F087843C5B2002D97
:1012900000F02281A2F12000C2B25808039044F26B
:1012A0001E7002EB4207C0F6000000EB470944F64F
:1012B000BA500197C0F60000049F4FF0000C00EBFD
:1012C000021002920090059308E000BF069D0CF109
:1012D000010C013D09F1010900F0FE80082B4E468A
:1012E0001ED0182B0CD0102B16D00C2B40F0F480F5
:1012F000019A44F64610C0F6000000EB820608E0B2
:10130000029A45F2AA3002EBC206C0F6000000EBDA
:101310008606664404E000BF009800EB0C0600BFA0
:1013200040F2180096F900B0FEB2CAB2C2F2000054
:10133000D20800EBC60801F0070418F8026001208B
:1013400000FA04F426EA040ADDF840E03443564685
:101350000695BEF1000F04BF264654465FEACB75E2
:1013600008BF344608F802404A1CD4B2E40802F030
:10137000070218F8045000FA02F225EA02062A438E
:101380003546BEF1000F04BF154632465FEA8B7644
:1013900058BF2A4608F804208A1CD4B2E40802F098
:1013A000070218F8045000FA02F225EA02062A435E
:1013B0003546BEF1000F04BF154632465FEA4B7654
:1013C00058BF2A4608F80420CA1CD4B2E40802F028
:1013D000070218F8045000FA02F225EA02062A432E
:1013E0003546BEF1000F04BF154632465FEA0B7664
:1013F00058BF2A4608F804200A1DD4B2E40802F0B7
:10140000070218F8045000FA02F225EA02062A43FD
:101410003546BEF1000F04BF154632465FEACB6683
:1014200058BF2A4608F804204A1DD4B2E40802F046
:10143000070218F8045000FA02F225EA02062A43CD
:101440003546BEF1000F04BF154632465FEA8B6693
:1014500058BF2A4608F804208A1DD4B2E40802F0D6
:10146000070218F8045000FA02F225EA02062A439D
:101470003546BEF1000F04BF154632465FEA4B66A3
:1014800058BF2A4608F80420CA1DD4B2E40802F066
:10149000070218F8045000FA02F225EA02062A436D
:1014A00035463B46BEF1000F04BF15463246BBF140
:1014B000000F58BF2A46059B0137082B08F8042067
:1014C0003FF404AF049CFAB2039E121BB24204BF65
:1014D00027460831FAE600BF07B0BDE8F08F0000EC
:1014E0002DE9F04F85B00192DA0801275E0718BF99
:1014F00007EBD30202FB03FCBCF1000F0493039043
:1015000000F0128104981038C2B2400140EAD200C3
:10151000C3B2062B00F208814FF0010E0EFA03F061
:1015200010F0470F00F0008144F2F620019AC0F657
:10153000000000EB421944F29E40C0F6000000EBB0
:10154000C2100E9D0090039800270293D2E000BFC6
:10155000009AD61940F2180396F900A0C6B2CAB292
:10156000C2F20003D20803EBC60801F0070B18F81B
:1015700002600EFA0BF326EA030433432646002DDD
:1015800004BF1E4623465FEACA7408BF334608F804
:1015900002304A1CD3B2DB0802F0070218F80340FD
:1015A0000EFA02F224EA020622433446002D04BF5A
:1015B000144632465FEA8A7658BF224608F803206E
:1015C0008A1CD3B2DB0802F0070218F803400EFAB7
:1015D00002F224EA020622433446002D04BF1446D8
:1015E00032465FEA4A7658BF224608F80320CA1CF2
:1015F000D3B2DB0802F0070218F803400EFA02F239
:1016000024EA020622433446002D04BF1446324623
:101610005FEA0A7658BF224608F803200A1DD3B2B3
:10162000DB0802F0070218F803400EFA02F224EA7F
:10163000020622433446002D04BF144632465FEAB8
:10164000CA6658BF224608F803204A1DD3B2DB08F9
:1016500002F0070218F803400EFA02F224EA02062A
:1016600022433446002D04BF144632465FEA8A66A0
:1016700058BF224608F803208A1DD3B2DB0802F0C7
:10168000070218F803400EFA02F224EA0206224387
:101690003446002D04BF144632465FEA4A6658BFFE
:1016A000224608F80320CA1DD3B2DB0802F0070265
:1016B00018F803400EFA02F224EA020622433446E6
:1016C000002D04BF14463246BAF1000F58BF22461F
:1016D0000130039C08F80320C2B2049B121B9A42FB
:1016E00004BF08312046029B0137BCF1010C09F10F
:1016F000010919D0022B3FF42BAF012B08D0002B8E
:101700004E463FF427AF44F21E52C0F6000220E7D7
:10171000019A02EBC20644F25642C0F6000202EB06
:10172000C6063E4416E700BF05B0BDE8F08F0000D6
:101730002DE9F04F85B0002B049167D00E998246B9
:101740004D080220082908BF00EB5105981E0290A1
:1017500058421C4616464FF000095FFA80FB42F2E1
:101760001078039223E000BF0120B6FBF0F04CF6A6
:10177000CD41CCF6CC41A0FB0112D10801EB810197
:10178000A0EB410009FB05A140F03002002808BF92
:101790003022C8B20499DDE90E37D2B20097FFF7C4
:1017A00065FD09F101095FFA89F0A0422ED26FEAC6
:1017B0000900C1B25945D7D00299A1EB0901C9B2BC
:1017C000032900EB040101D2012009E001F0FC0231
:1017D000002301200433DEB2964200FB08F0F9D169
:1017E000039E11F00301C0D0012903D100EB80005A
:1017F0004000BAE74FF47A72424302294FF0640185
:1018000008BF00FB01F21046AFE700BF05B0BDE81E
:10181000F08F00002DE9F04F82B0DF085D070092E5
:101820004FF0010618BF06EBD307002F00F0E18050
:1018300084460098002800F0DC800B9C0098A4F1FE
:10184000010A00FB07F366464FF001090120012B56
:1018500098BF034640F218020193F7B2CBB2C2F22E
:10186000000260464FEAD30C02EBC70701F0070401
:1018700017F80C5009FA04F4DDF830E01AF901BF4A
:1018800025EA04082C43BEF1000F454604BF254657
:1018900044465FEACB7301F1010308BF2C46DDB279
:1018A00007F80C40ED0803F007037C5D09FA03F329
:1018B000844624EA03002343BEF1000F024604BF1E
:1018C0001A4603465FEA8B7001F1020058BF1346C7
:1018D000C2B27B55D20800F00700BB5C09FA00F0E9
:1018E00023EA000518432B46BEF1000F04BF034650
:1018F00028465FEA4B7558BF1846B854C81CC2B298
:10190000D20800F00700BB5C09FA00F023EA0005EA
:1019100018432B46BEF1000F04BF034628465FEA7A
:101920000B7558BF1846B854081DC2B2D20800F053
:101930000700BB5C09FA00F023EA000518432B46B8
:10194000BEF1000F04BF034628465FEACB6558BFCF
:101950001846B854481DC2B2D20800F00700BB5C5C
:1019600009FA00F023EA000518432B46BEF1000FE8
:1019700004BF034628465FEA8B6558BF1846B85433
:10198000881DC2B2D20800F00700BB5C09FA00F063
:1019900023EA000518432B46BEF1000F04BF03469F
:1019A00028465FEA4B6558BF1846B854C81DC2B2F6
:1019B000D20800F00700BB5C09FA00F023EA00053A
:1019C00018432B46BEF1000F04BF034628460136DC
:1019D000BBF1000F58BF1846F3B2009DA3EB0C03F8
:1019E000AB42019B04BF66460831013BB8547FF40B
:1019F00031AF02B0BDE8F08F2DE9F04381B09946D8
:101A000013780D46A3F12001C9B25E291BD8DDF879
:101A1000208006464FEA5907541EB9F1080F08BF47
:101A2000062700BFF0B2DAB229464B46CDF8008057
:101A3000FFF71CFCA3783E44A3F12000C0B25F284E
:101A400004F10104EED301B0BDE8F0832DE9F04FBD
:101A500087B0DDF84480059010469A460C46029205
:101A6000FEF7F8FB83464FEA5800BAF1000F0690E4
:101A7000049457D0AAF102000390CAF10000002795
:101A8000C5B242F210791FE00120BBFBF0F04CF62A
:101A9000CD41CCF6CC41A0FB0112D10801EB810174
:101AA000A0EB4100DDE90521129E07FB012140F07A
:101AB0003002C8B2D2B2214643460096FFF7D6FBA9
:101AC0000137F8B250452DD2F843C1B2A942DBD05C
:101AD0000399C91BC9B2032900EB0A0102D20120F4
:101AE0000AE000BF01F0FC02002301200433DCB255
:101AF000944200FB09F0F9D1049C11F00301C4D019
:101B0000012903D100EB80004000BEE74FF47A7258
:101B1000424302294FF0640108BF00FB01F2104666
:101B2000B3E700BFDDE90510129F00FB0A10214654
:101B3000C0B22E2243460097FFF798FB5846FEF7A7
:101B40007BFB01460298FEF73FFB109D002D00F045
:101B500095800646681E0390C0B2032805F0030175
:101B600002D20A22A1B91DE005F0FC0200230120E7
:101B700042F2107704330546D8B2904205FB07F0D5
:101B8000F8D148F2A062C0F201026A43109D49B147
:101B9000012906D0642302EB82005A43022908BFC0
:101BA00042001046FEF751FB01463046FEF712FB9D
:101BB000FEF750FB002D61D0064605984FF0000B54
:101BC00000F10508A81E059068425FFA80F942F20C
:101BD000107523E00120B6FBF0F04CF6CD41CCF6B9
:101BE000CC41A0FB0112D10801EB8101069AA0EBC8
:101BF00041000BEB0A0101FB028140F03000DDE9FE
:101C00001137C2B2C8B221460097FFF72FFB0BF184
:101C1000010B10995FFA8BF088422FD26FEA0B000C
:101C2000C0B24845D6D00598A0EB0B00C0B203283F
:101C30000398A0EB0B0101D2012009E001F0FC02A6
:101C4000002301200433DCB2944205FB00F0F9D1FB
:101C5000049C11F00301BED0012903D100EB8000E8
:101C60004000B8E74FF47A72424302294FF0640112
:101C700008BF00FB01F21046ADE700BF07B0BDE8AA
:101C8000F08F0000B0B582B00446002001902168BA
:101C90008A68D2074FD1886840F00100886040F21E
:101CA0001000C2F2000000684DF68361C4F21B31DF
:101CB000A0FB0101880C01900198A0B101980138A6
:101CC0000190019878B1019801380190019850B1C4
:101CD000019801380190019828B1019801380190CC
:101CE00001980028EAD100F07FFD21688968C907C2
:101CF0001CD1054603E000BF8068C0071AD100F080
:101D000073FD411B20680329F6D38168C907F3D10D
:101D1000A06A40F01000A062E06A40F00100E062BA
:101D2000002084F82400012002B0B0BD002002B0E1
:101D3000B0BD00BF002002B0B0BD0000FEE7000053
:101D400070B540F2413141F29112C0F60001C0F687
:101D50000002C0E9081241F6F91140F28D73C0F695
:101D6000000141F2E14241F2317441F64D2541F664
:101D7000150640F62D1C40F6710EC0F60003C0F6A5
:101D80000002C0F60004C0F60005C0F6000680E8B8
:101D9000320000F10C01C0F6000CC0F6000E81E824
:101DA0000450C0E90636FEF7D9FD70BD704700004B
:101DB000EFF3108072B600BFFEE7000010B581B0EF
:101DC0000022009290F82420012A03D10221084623
:101DD00001B010BD4B680122062B80F8242017D8D3
:101DE000D0F800C003EB83035A1F1F23DCF834E054
:101DF00003FA02F40B682EEA040403FA02F2224307
:101E0000CCF83420092B03EB430219D936E000BF8C
:101E1000D0F800C00C2B03EB83021DD8233A1F23FC
:101E2000DCF830E003FA02F40B682EEA040403FA4B
:101E300002F22243CCF83020092B03EB43021DD8D9
:101E4000DCF81030072489689440A343914019437B
:101E5000CCF81010002130E0413A1F23DCF82CE0D0
:101E600003FA02F40B682EEA040403FA02F2224396
:101E7000CCF82C20092B03EB4302E1D9DCF80CE071
:101E80001E3A0724896894402EEA0404914023F006
:101E900001022143102ACCF80C100DD142F2084166
:101EA000C4F20101A1F1080294450DD0816A41F00C
:101EB00020018162012100E00021002280F824201D
:101EC000084601B010BD00BF0A68120230D40A688B
:101ED000102B42F400020A602CD140F21001C2F231
:101EE000000109684DF68362C4F21B32A1FB0212A5
:101EF000910C01EB8101490000910099E1B1009939
:101F0000013900910099C9B10099013900910099F6
:101F1000B1B1009901390091009999B10099013945
:101F20000091009900294FF00001E8D1C5E700BFFA
:101F30000021C2E70021C0E70021BEE70021BCE785
:101F40000021BAE70021B8E7806A70470068C06CDA
:101F500070470000B0B5002800F0A8800446806AF1
:101F600020B121688868C0070BD114E00020E0622E
:101F700084F82400204600F09BF821688868C00798
:101F800009D0886820F00100886000F02DFC2168ED
:101F90008A68D20726D1A06AC0063AD4A06A41F264
:101FA000021290430230A062E069D4E9013240EAB3
:101FB000030C531EB3FA83F35D091346B2F5807F19
:101FC00018BF2B02207D257B01284CEA450030D12B
:101FD00035B3A56A45F02005A562E56A45F001051F
:101FE000E56226E0054602E08868C007D3D000F02D
:101FF000FBFB401B21680328F6D38868C007F3D099
:10200000A06A40F01000A062E06A40F00100E062C7
:10201000A06AA06A40F01000A0620120B0BD00BF1D
:10202000D4F818C04EF60005CFF6FF7505EB4C3519
:102030002B434D68B2F5807F25F4694543EA0503DB
:102040004B608B684FF2FD75CFF6E17503EA05032F
:1020500043EA00038B6001D0012A07D122690023E3
:10206000CFF6F07303EB025201E000BF0022CB6A0F
:1020700023F470031A43CA62896840F6FE62CFF601
:102080001F721140814207D10020E062A16A012243
:1020900062F30101A162B0BDA06A40F0100020F01F
:1020A0000200A062E06A40F00100E0620120B0BDE1
:1020B00080B586B0014640F60040C4F201000968D0
:1020C00000F5C05291424FF00001CDE9041101D05A
:1020D00006B080BD41F21801C4F202010A6842F460
:1020E00000720A600A6802F400720192019A0A689A
:1020F00042F008020A60096801F0080101910199A3
:102100000321CDE9021102A900F05AFA06B080BD00
:10211000F0B581B000270D460446009700F064FB3F
:1021200021688A68D20543D406464868C00503D4AE
:10213000C86A10F4700F45D040F21000C2F20000DF
:102140000768022000F00EFC216844F624130A6997
:10215000B7FBF0F0C2F292431A4206D1CA6844F6C5
:102160002413C0F292031A425ED00A6942F29243EB
:10217000C1F249231A4207D1CA6842F29243C0F21F
:1021800049031A4200F0C0800A6949F24923C0F2AB
:1021900024031A424FF0FC0257D1CF681F4208BFF8
:1021A0005422009B02FB00F7BB4253D3C3E000BFA5
:1021B000A06A40F02000A06284F82470012001B0E1
:1021C000F0BD00BF0868800700F1B580681C00F012
:1021D000A880FDB90868800772D50868800700F1FB
:1021E000AA80086880076BD50868800700F1A38083
:1021F0000868800764D50868800700F19C8008683B
:1022000080075DD508688007E4D594E008688007FA
:1022100000F1918000F0E8FA801B2168A842F5D90E
:1022200008688007F2D44BE00A6942F29243C1F297
:1022300049231A424FF0290207D1CB6842F2924754
:10224000C0F249073B4208BF1422009B02FB00F783
:10225000BB4270D2681C4FD055BB0098B8422FD3F8
:102260000098013000900098B84264D20098B842BB
:1022700026D30098013000900098B8425BD20098B5
:10228000B8421DD30098013000900098B84252D255
:102290000098B84214D30098013000900098B842DA
:1022A000DBD348E00098013000900098B84233D268
:1022B00000F09AFA801BA842F4D90098B842F1D2F3
:1022C000A06A40F00400A062002084F824000320EB
:1022D00001B0F0BD0098013000900098B8422AD2B9
:1022E0000098013000900098B84224D20098013044
:1022F00000900098B8421ED20098013000900098DB
:10230000B842E7D317E000BF5422009B02FB00F75E
:10231000BB429FD30FE000BF21680CE00868800734
:1023200009D40868800706D4086880075CBF08687D
:102330005FEA8070F2D56FF012000860A06A40F486
:102340000070A062886800F46020B0F5602F01D1B1
:10235000207B18B1002001B0F0BD00BFA06A20F4BE
:102360008070A062A06AC004F4D4A06A40F00100AA
:10237000A062002001B0F0BD10B5044690F8240022
:10238000012804BF022010BD012084F8240020464B
:10239000FFF778FC20B1002184F8241010BD00BFA5
:1023A00042F2044C2068A16AC4F2010C40F20132EE
:1023B00091430CF57F7201F580719042A16233D098
:1023C000A16A21F48011A1624168490504D5A16A7E
:1023D000012363F30D31A162A16A0023C9044FF008
:1023E000000144BFE16A21F00601E1626FF00201E1
:1023F00084F824300160816801F46021B1F5602F18
:1024000006D190420AD1DCF8001011F4702F05D0EB
:10241000816841F480118160002010BD816841F421
:10242000A0018160002010BDDCF8001011F4702FB5
:10243000C6D0A16A41F48011A162DCF80010490500
:10244000C5D4C9E7B0B5044690F82400012804BFFC
:102450000220B0BD0121206884F824108168C907DA
:1024600009D0816821F00101816000F0BDF9216887
:102470008968C9070ED1214651F8280F41F201128F
:1024800020EA0202002042F001020A60002184F8E2
:102490002410B0BD054602E08068C007EBD000F014
:1024A000A3F9411B20680329F6D38168C907F3D03B
:1024B000A06A214640F01000A06251F82C2F0120A4
:1024C000E1E70000014690F82100022816D10868D3
:1024D000D1E90FC3026822F00E020260026822F006
:1024E00001020260012000FA03F2CCF8042081F816
:1024F00021000020002281F82020704704208863FA
:102500000120002281F820207047000080B590F85B
:102510002110022924D10268116821F00E011160F6
:102520002F211368C4F202018A4240F20401C4F26E
:10253000020123F00103136016DD3023C4F202030D
:102540009A421DD04423C4F202039A421CD058235D
:10255000C4F202039A421DD14FF4803322E000BF3F
:1025600004218163012080BD0823C4F202039A4242
:102570000ED01C23C4F202039A420BD1102311E0A7
:102580004FF480730EE000BF4FF480530AE000BFA9
:10259000012307E001F1680C4FF08073624508BF2A
:1025A0004FF480130B60012180F82110426B002151
:1025B00080F820100AB190470021084680BD000035
:1025C0002DE9F04F82B00E68002E00F0038141F239
:1025D0000042C4F20102042340F2004E904208BFC0
:1025E00003234FF6FF7CC4F2010E00930024012365
:1025F000C1F2100C4FF0000A4FF0000949E000BF93
:10260000012704F00C030F229A402BEA020207FA7A
:1026100003F34FEA9A051A4346F82520D1F804B08F
:1026200040F20C455FEACB22DEF8082054BF22EAD4
:10263000080242EA0802C4F20105CEF808202A681E
:102640005FEA8B2354BF22EA080242EA08022A60AA
:102650005FEA8B33DEF8042054BF22EA080242EA24
:1026600008025FEACB33CEF80420DEF800204FF0FA
:10267000010354BF22EA080242EA0802CEF8002011
:102680000E680AF1010A36FA0AF204F1040400F0B5
:10269000A18003FA0AF816EA080FF1D04E686645E1
:1026A00012DC122E56D8DFE806F0350B4549555599
:1026B00055555555555555555555554D510000BF16
:1026C000D1F80C9046E000BF4FF6FF72C1F2210234
:1026D00096420FDC0022C1F2110296421AD000226B
:1026E000C1F21202964215D00022C1F22102964296
:1026F00010D02FE00022C1F2220296420AD000221E
:10270000C1F23102964205D00022C1F23202964255
:1027100020D100BF8A684AB1012A14BFC0F81480D2
:10272000C0F810804FF0080914E000BF4FF0040912
:1027300010E000BFCA6802F108090BE04FF0000981
:1027400008E000BFCA6802F1040903E0CA6802F1A8
:102750000C0900BF22460646BAF1080F24BF203AF2
:10276000043637680F25954027EA050509FA02F275
:102770002A433260CA79D2067FF582AF41F218034C
:10278000C4F202031A68AEF57E7642F001021A60C6
:102790001A6802F001020192019A2AF0030256F827
:1027A00002B040F60002C4F20102904210D040F69E
:1027B0000042C4F2010290423FF422AF41F2000213
:1027C000C4F20102009F904208BF022719E700BF30
:1027D000002716E702B0BDE8F08F0000002A08BF0E
:1027E000090401617047000040F2A850C2F20000E5
:1027F0000068704740F2000040F2A851C2F20000A9
:10280000C2F2000100780A681044086070470000B6
:1028100080B542F20000C4F20200016841F01001EC
:102820000160032000F08EF80F2000F005F800F0A2
:1028300027F8002080BD000070B540F20006C2F20B
:10284000000640F210013278C2F200014FF47A73B0
:102850000968B3FBF2F20446B1FBF2F1084600F05E
:10286000E7FD0F2C4FF0010508D838B94FF0FF30C5
:1028700021460022002500F039F87460284670BD1A
:1028800082B041F21800C4F202000168022241F055
:1028900001010160016801F00101019101994168A4
:1028A00041F080514160406800F0805000900098F5
:1028B0000420C4F20100016862F31A61016002B0F1
:1028C00070470000002848BF7047C1B200F01F00E9
:1028D000012202FA00F04EF20012CEF2000242EAA9
:1028E000D10121F0030108607047000010B54EF6D9
:1028F0000C5CCEF2000CDCF80030C3F3022E8EF03C
:102900000704042C28BF0424BEF103034FF0FF3E4C
:102910000EFA04F438BF0023A14399400EFA03F3E2
:102920009A43114300F00F0200F160430901043A99
:1029300003F564436244002848BF02F10C03197098
:1029400010BD00004EF60C51CEF200010A684FF6A1
:10295000FF031A4060F30A2242F0806040F0FD70ED
:102960000860704780B5012818D0022836D010289A
:1029700032D141F20401C4F202010A6851F8040C98
:10298000C00129D5C2F383402DA3185CD2033DD4E6
:1029900040F60012C0F23D02504343E041F2040011
:1029A000C4F20200C16940F202320A40B2F5817FEE
:1029B00004BF4FF4004080BD01F44071B1F5407F89
:1029C0001CD0B1F5007F07D1006A49F6404180076D
:1029D00001EAE07080BD00BF002080BD00F0B4F9C6
:1029E00041F20401C4F2020109680222C1F38131FB
:1029F00002EB4101B0FBF1F080BD00BF50F8040CC8
:102A00004FF22441800301EAE07080BD0A6810A300
:102A1000C2F340429A5C41F20023C0F27A03B3FB56
:102A2000F2F250430968490248BF80BD4AF6AB2123
:102A30004000CAF6AA21A0FB0101480880BD00BFE2
:102A400002030405060708090A0B0C0D0E0F1010EF
:102A5000010200002DE9F04182B00446007841F205
:102A60001C06C007C4F202064AD0306810F0805835
:102A700008D1306840F080503060306800F08050FD
:102A80000190019847F20007C4F200073868C005BA
:102A900012D4386840F480703860FFF7A5FE054610
:102AA0003868C00508D4FFF79FFE401B6428F7D99B
:102AB000032002B0BDE8F081706810F4407012D0BD
:102AC000616801F4407188420DD0706840F2404264
:102AD000C4F24222012320F4407113600023C00796
:102AE000136071602AD17068616820F440700843F7
:102AF000B8F1000F706003D1306820F08050306072
:102B00002068810707D556F8181CA26821F44041B7
:102B1000114346F8181CC00604D4002002B0BDE8DA
:102B2000F08100BF56F8180CE16820F480000843DB
:102B300046F8180C002002B0BDE8F081FFF754FE03
:102B4000054641F2883700BF70688007CBD4FFF795
:102B50004BFE401BB8424FF00300F5D9EBE70000F5
:102B60002DE9F04381B0002800F0858042F2000892
:102B7000C4F202080446D8F800000D4600F0070031
:102B800088420CD2D8F8000020F007002843C8F88B
:102B90000000D8F8000000F00700A8426BD12068C0
:102BA00041F204098107C4F2020917D5410705D58E
:102BB000D9F8001041F4E061C9F80010010705D50B
:102BC000D9F8001041F46051C9F80010D9F800108C
:102BD000A26821F0F0011143C9F80010C00741D1EB
:102BE000D8F8000000F00700A8420CD9D8F800007F
:102BF00020F007002843C8F80000D8F8000000F0D3
:102C00000700A84237D12068410707D5D9F800103E
:102C1000E26821F4E0611143C9F80010000708D50B
:102C2000D9F80000216920F4605040EAC100C9F8D9
:102C30000000D9F8002002F00C00082841F2002022
:102C4000C0F27A0050D146F20613C2F38341C0F6B7
:102C50000003595CD2033BD440F60010C0F23D00A3
:102C6000484341E0606802280AD001282AD159F877
:102C7000041C890308D4012001B0BDE8F08300BF23
:102C800059F8041C8901F6D5D9F8001021F0030188
:102C90000843C9F80000FFF7A7FD064641F2883750
:102CA000D9F80000616800F00C00B0EB810F97D0FC
:102CB000FFF79AFD801BB842F2D9032001B0BDE8AE
:102CC000F08300BF59F8041C8907D4D5DCE700BFA6
:102CD000D9F8002044F2F423C2F34042C0F60003C6
:102CE0009A5C4843B0FBF2F0D9F8001044F2DC22C1
:102CF000C1F30311C0F60002515C40F2100220FA49
:102D000001F140F20400C2F200000068C2F20002C9
:102D10001160FFF791FD002001B0BDE8F0830000D5
:102D200040F2100041F20401C2F20000C4F20201BC
:102D30000068096844F2EC22C1F30221C0F60002E7
:102D4000515CC8407047000040F2100041F204019D
:102D5000C2F20000C4F202010068096844F2EC22E9
:102D6000C1F3C221C0F60002515CC84070470000A8
:102D70002DE9F04182B0002868D00446007841F285
:102D80000006C007C4F2020625D0706800F00C00EF
:102D900004281BD0706800F00C00082802D170686D
:102DA000C00313D46068002800F06881B0F5A02F3C
:102DB00000F07C81B0F5803F00F07C81306820F429
:102DC00080303060306820F4802076E13068800305
:102DD00001D56068D0B32078800718D5706810F0EE
:102DE0000C0F07D0706800F00C0008286ED17068D6
:102DF000C0036BD43068800702D52069012825D133
:102E00003068616920F0F80040EAC1003060207845
:102E100000071FD42078400732D4E56995B1706867
:102E200000F00C00082840F08F80012D0ED0706853
:102E3000216A00F480328A4208D1616A00F470107D
:102E4000884203D1002002B0BDE8F081012002B029
:102E5000BDE8F081A069002862D00020C4F24220C1
:102E60000121C0F88014FFF7BFFC0546706A800797
:102E700000F18C80FFF7B8FC401B0228F6D92AE14C
:102E8000F06910F0805808D1F06940F08050F0618E
:102E9000F06900F080500090009847F20007C4F2FB
:102EA00000073868C00529D4386840F4807038605D
:102EB000FFF79AFC054600BF3868C0051ED4FFF72F
:102EC00093FC401B6428F7D905E100BF2069002866
:102ED00040F20000C4F2422000F082800121016033
:102EE000FFF782FC054600BF306880073FF588AFDA
:102EF000FFF77AFC401B0228F6D9ECE0E0680028D6
:102F000000F08080052800F09780012800F098806C
:102F1000306A20F001003062306A20F0040092E054
:102F20000020C4F242200021C0F88014FFF75CFCAE
:102F3000054600BF706A80077FF56CAFFFF754FC51
:102F4000401B0228F6D9C6E00027C4F24227002021
:102F50003866FFF749FC022D05460BD13068800129
:102F600040F1BE80FFF740FC401B02284FF00300F9
:102F7000F4D968E7306880017FF564AFFFF734FC6F
:102F8000401B02284FF00300F4D95CE740F2100028
:102F9000C2F20000006844F6D351C1F26201A0FB06
:102FA0000101480A019000BF00BF0198411E00289E
:102FB00001913FF42FAF00BF0198411E00280191FD
:102FC0003FF428AF00BF0198411E002801913FF453
:102FD00021AF00BF0198411E00280191E4D119E7FB
:102FE00000210160FFF700FC054600BF3068800744
:102FF0007FF50DAFFFF7F8FB401B02284FF00300F1
:10300000F4D920E7306A20F001003062306A20F005
:1030100004003062FFF7E8FB054641F2883700BF45
:10302000306A800720D5FFF7DFFB401BB8424FF026
:103030000300F5D907E700BF306A40F004003062B2
:10304000306A40F001003062FFF7CEFB054641F2E6
:10305000883700BF306A800706D4FFF7C5FB401BE6
:10306000B842F7D937E000BFB8F1000F7FF4D5AE12
:10307000F06920F08050F061CFE600BF306820F4A6
:1030800080303060306820F480203060FFF7ACFB87
:10309000054600BF306880037FF59DAEFFF7A4FBB7
:1030A000401B64284FF00300F4D9CCE6306840F4AC
:1030B00080203060306840F480303060FFF794FB4F
:1030C000054600BF306880033FF585AEFFF78CFBF7
:1030D000401B6428F6D9032002B0BDE8F08100BF90
:1030E000206AB0F5803F05D17168A26821F40031F3
:1030F000114371607168626A21F4741111430843CD
:10310000706001203866FFF76FFB0446306880016D
:103110003FF598AEFFF768FB001B02284FF0030055
:10312000F4D990E670B538B10446406A30B1002059
:10313000206104F1140007E0012070BD6068B0F563
:10314000827F03D004F11C00002101600026A662EA
:1031500094F8510020B9204684F8506000F038F807
:10316000022084F8510094E8071001F4827103688A
:1031700002F4044223F040030360236911440CF479
:103180000062114403F002026369114403F001027A
:10319000A369E569114403F40072114405F0380293
:1031A000256A114405F08002A56A114305F4005216
:1031B00011430160042101EA13414160C16921F416
:1031C0000061C1610120666584F85100304670BD20
:1031D00080B586B043F600010068C4F20001002209
:1031E0008842049202D006B080BD00BF41F21800B0
:1031F000C4F20200426842F480424260426802F433
:1032000080420192019A026842F00802026000685E
:1032100000F00800019001984FF420400290022035
:1032200003900320059001F5544002A9FFF7C8F967
:1032300006B080BD2DE9F04182B0044690F8500000
:10324000012803D1022002B0BDE8F08101201D4613
:1032500016460F4684F85000FFF7C6FA94F851104E
:1032600001290DD18046002F4FF0010018BF002E1C
:103270000ED1002184F8501002B0BDE8F08100BFEB
:103280000220002184F8501002B0BDE8F08100BF98
:103290000320002184F8510061652763A686E68635
:1032A000A163A187E187A0682164B0F5004F206881
:1032B000616407D1016821F040010160016841F4B7
:1032C000804101600168490603D4016841F0400172
:1032D00001606168731EE268B1FA81F1B3FA83F3A9
:1032E00049095B09B2F5006F41EA03013CD131B1F4
:1032F00037F8021BC1602763E08E0138E086E08E5C
:1033000000286BD0681C0CD11DE000BF216B31F888
:10331000022BC2602163E08E0138E086E08E002837
:103320005CD0206881688907F0D4FFF75DFAA0EBD4
:103330000800A842F2D3032071E000BFFFF754FA5F
:10334000E08E00284AD0206881688907F6D5216B75
:1033500031F8022BC2602163E08E0138E086E08EF6
:103360000028F0D13AE000BF39B139780173206B01
:1033700001302063E08E0138E086E08E70B3681C77
:103380000BD11BE0216B09780173206B01302063A6
:10339000E08E0138E086E08E00B3206881688907FE
:1033A000F0D4FFF721FAA0EB0800A842F3D30320E2
:1033B00035E000BFFFF718FAE08E78B12068816829
:1033C0008907F7D5216B09780173206B01302063E1
:1033D000E08E0138E086E08E0028EFD12046802183
:1033E0002A46434600F0AEFD28B1606D40F0200053
:1033F000606520206065A06838B9002001902068D1
:10340000C1680191806801900198606D30B1012020
:10341000002184F8501002B0BDE8F08100200121A5
:1034200084F85110002184F8501002B0BDE8F081FA
:10343000411E0020B0EB116F1CBF012070474EF2FF
:103440001002CEF2000251604EF62351CEF200017E
:10345000F0230B70072190601160704770470000E7
:1034600070470000B0B582B0044600680168C368C8
:10347000426901F02F05202D03F0200506D12DB162
:10348000204602B0BDE8B04000F0DABD5FEA017C42
:103490001EBF02F0010E03F4907212EB0E0253D124
:1034A000226B012A05D111F0100218BF13F010028F
:1034B00036D10A0622D513F080021FD094F84110AD
:1034C00021293FD1A168B1F5805F03D1216900298D
:1034D00000F07082216A4A1C226209784160E18C06
:1034E00001390A04E1842DD1C16821F08001C16055
:1034F000C16841F04001C16002B0B0BD490621D5AC
:1035000013F040011ED0C16821F04001C1602021AC
:10351000204684F8411002B0BDE8B04000F00CBB7A
:10352000002101910168019141680191019940696F
:10353000400613D4A08DE18DE28D002A18BF884289
:1035400040F0BA8102B0B0BDCA0718BF13F4807250
:1035500040F0B6804A0700F1B980BEE0E06B016838
:1035600049688AB2002AEDD0A38D9A42EAD2E18559
:103570008069202800F09C80206850E8030F2168B3
:1035800020F4807041E80302DAB1206850E8030FAC
:10359000216820F4807041E8030292B1206850E86D
:1035A000030F216820F4807041E803024AB12068CB
:1035B00050E8030F216820F4807041E80302002ADC
:1035C000DAD1206850E8050F216820F0010041E8B9
:1035D0000502DAB1206850E8050F216820F00100EB
:1035E00041E8050292B1206850E8050F216820F0FB
:1035F000010041E805024AB1206850E8050F216842
:1036000020F0010041E80502002ADAD1206850E8E4
:10361000050F216820F0400041E80502DAB120687A
:1036200050E8050F216820F0400041E8050292B102
:10363000206850E8050F216820F0400041E80502AD
:103640004AB1206850E8050F216820F0400041E8A9
:103650000502002ADAD1202084F8420000202063ED
:10366000206850E8030F216820F0100041E80302B1
:10367000DAB1206850E8030F216820F0100041E81B
:10368000030292B1206850E8030F216820F0100077
:1036900041E803024AB1206850E8030F216820F096
:1036A000100041E80302002ADAD1E06BFEF70AFFBE
:1036B00002206063A08DE18D401A81B2204674E142
:1036C000626C42F0010262644A0706D5BEF1000F47
:1036D00003D0626C42F0020262648A0706D5BEF132
:1036E000000F03D0626C42F004026264BCF1000F70
:1036F00009D545EA0E02B2FA82F2520903D1626C90
:1037000042F008026264626C002A3FF41BAF11F0C1
:10371000200118BF002D03D0204600F091FC206846
:103720004069616C00F0400001F00801401800F0B1
:10373000B58000BF206850E8030F216820F4907026
:1037400041E80302BAB3206850E8030F216820F46F
:10375000907041E8030272B3206850E8030F2168BB
:1037600020F4907041E803022AB3206850E8030F68
:10377000216820F4907041E80302002ADAD11AE0AF
:10378000206850E8050F216820F0010041E805029B
:10379000DAB1206850E8050F216820F0010041E807
:1037A000050292B1206850E8050F216820F0010061
:1037B00041E805024AB1206850E8050F216820F071
:1037C000010041E80502002ADAD1206B012824D14A
:1037D000206850E8030F216820F0100041E8030240
:1037E000DAB1206850E8030F216820F0100041E8AA
:1037F000030292B1206850E8030F216820F0100006
:1038000041E803024AB1206850E8030F216820F024
:10381000100041E80302002ADAD1202084F8420097
:10382000002020632068406940063FD5206850E8AA
:10383000050F216820F0400041E80502DAB1206858
:1038400050E8050F216820F0400041E8050292B1E0
:10385000206850E8050F216820F0400041E805028B
:103860004AB1206850E8050F216820F0400041E887
:103870000502002ADAD1E06BC0B144F23501C0F68E
:1038800000014163FEF742FE00283FF45BAEE06BAF
:10389000416B02B0BDE8B040084700BF2046FFF7CB
:1038A000DFFD0020606402B0B0BD00BF204602B062
:1038B000BDE8B040FFF7D4BD401A216851E8031FAE
:1038C000226821F4907142E80313DBB1216851E8CA
:1038D000031F226821F4907142E8031393B1216819
:1038E00051E8031F226821F4907142E803134BB1A1
:1038F000216851E8031F226821F4907142E8031304
:10390000002BDAD1216851E8051F226821F001015E
:1039100042E80513DBB1216851E8051F226821F058
:10392000010142E8051393B1216851E8051F22689F
:1039300021F0010142E805134BB1216851E8051F50
:10394000226821F0010142E80513002BDAD1202181
:1039500084F8421000212163216851E8031F226886
:1039600021F0100142E80313DBB1216851E8031F85
:10397000226821F0100142E8031393B1216851E855
:10398000031F226821F0100142E803134BB12168A4
:1039900051E8031F226821F0100142E80313002BB5
:1039A000DAD1022281B22046626302B0BDE8B040A3
:1039B000FFF754BD216A31F8022B6FF35F2242609A
:1039C00021628CE5002804BF0120704710B5044631
:1039D00090F8410028B9002084F84000204600F00B
:1039E00063F8242084F841002068D4E90212C368F7
:1039F00023F40053C360036923F440531A43026164
:103A0000D4E904231143C268194341F20C639A4379
:103A10001143C1604169A26921F44071114343F629
:103A20000002C4F201029042416103D0FFF778F92D
:103A300002E000BFFFF788F962681921484391004E
:103A4000B0FBF1F048F21F51C5F2EB11A0FB0123CE
:103A50005A094FF69C73C0F6FF7302FB0300322332
:103A600003EB0010A0FB0101F02303EA51132068CF
:103A700003EB0212C1F3431111448160016921F487
:103A800090410161416921F02A014161C16841F41D
:103A90000051C16000202021606484F8411084F846
:103AA0004210606310BD000070B586B040F600049F
:103AB000C4F20104006804F54051002688420496CF
:103AC00002D006B070BD00BF41F21800C4F202007F
:103AD000016802AD41F480410160016801F4804158
:103AE00001910199016841F00401016000682946D3
:103AF00000F00400019001984FF400700290022041
:103B00000390032005902046FEF75AFD4FF4806095
:103B1000CDE90206204629460496FEF751FD2520F0
:103B200000210022FEF7E2FE2520FEF7CBFE06B0C4
:103B300070BD00007047000070470000FEE7000005
:103B40004FF0FF31C0E914110021A0F85810704760
:103B500010B584B040F2D84042F20041C2F20000F9
:103B6000C4F201014FF4807C002301244FF4602251
:103B700080E80A10022103730475C0E9064201615E
:103B8000FEF7E8F9002818BFFEF712F90920CDE981
:103B900001040720039040F2D840C2F2000001A9BE
:103BA000FEF70CF9002818BFFEF702F90820019073
:103BB0000220029040F2D840C2F2000001A9FEF7B4
:103BC000FDF8002818BFFEF7F3F804B010BD0000A0
:103BD0002DE9F04784B041F21800C4F202000168F8
:103BE00040F6004A41F0100101600168C4F2010A88
:103BF00001F010010091009901680AF5806541F01B
:103C0000200101600168002201F02001009100996B
:103C100001684FF4804641F00801016001684FF0EF
:103C2000000901F0080100910099016841F00401C8
:103C3000016000684FF4804100F00400009000989B
:103C40002846FEF7CBFD50464FF4A04100224FF42A
:103C5000A048FEF7C3FD00966E46012702242846C1
:103C60003146CDE901790394FEF7AAFC504631466E
:103C7000CDE90087CDE90294FEF7A2FC04B0BDE8CF
:103C8000F087000080B540F2085043F60001C2F210
:103C90000000C4F200014FF4827200234FF4007C54
:103CA00080E80E000A21C0E90333C0E9053CC36186
:103CB000C0E90833C0E90A31FFF734FA002808BF29
:103CC00080BDBDE88040FEF773B8000080B540F2CB
:103CD000605043F60001C2F20000C4F2010100236B
:103CE0004FF00C0C4FF4E13280E80E00C0E90333D2
:103CF000C0E905C3C361FFF765FE002808BF80BDAA
:103D0000BDE88040FEF754B8FEE70000FEE7000083
:103D10007047000080B540F21840C2F20000FFF783
:103D20000FFF40F27440C2F20000BDE88040FFF790
:103D300007BF00002DE9F04140F2D844C2F2000470
:103D40002046FEF719FB20460A21FEF7E1F920463E
:103D5000FEF7FAF840F208088005C2F2000816D50E
:103D600040F2D840C2F20000FEF7F0F8D8F8001098
:103D700004460846214600F001FA18B9D8F80000B8
:103D800000F0E6F9D8F80000214600F0F7F940F21B
:103D9000D844C2F200042046FEF7EEFA20460A217B
:103DA000FEF7B6F92046FEF7CFF8800516D540F2AB
:103DB000D840C2F20000FEF7C9F8D8F80410044653
:103DC0000846214600F0DAF918B9D8F8040000F0E6
:103DD000BFF9D8F80400214600F0D0F940F2D840ED
:103DE000C2F20000FEF72EFBD8F800E0BEF8580043
:103DF00050B1421E032A00F0030C07D20026002314
:103E0000BCF1000F1BD129E02DE000BF20F003031F
:103E1000AEF110045E420025002300BF54F8107F6D
:103E2000043D3B44D4E90172E1683B441A44AE428C
:103E300001EB0203F2D16E42BCF1000F0ED05EF82E
:103E40002650BCF1010F2B4408D00EEB86014E68C2
:103E5000BCF1020F33441CBF89680B44C0B2B3FBF2
:103E6000F0F0FCF7F2F9D8F804E040F2D048BEF8E0
:103E70005810C2F20008C8F8000059B1481E0328C3
:103E800001F0030C0AD200270023BCF1000F1ED161
:103E90002CE000BFC8F80400BDE8F08121F0030366
:103EA000AEF110055E420027002300BF55F8104F09
:103EB000043F2344D5E90140EA6823441844BE4244
:103EC00002EB0003F2D17F42BCF1000F0ED05EF88E
:103ED0002700BCF1010F034408D00EEB87025068A5
:103EE000BCF1020F03441CBF90680344C8B2B3FB8B
:103EF000F0F0FCF7AAF9C8F80400BDE8F081000072
:103F0000B0B5FFF717FF40F2D045C2F20005D5E982
:103F100000040021C3F64851FCF75CF90021CCF203
:103F2000C821FCF7FFF800212860C3F6C8512046DD
:103F3000FCF750F90021CCF24831FCF7F3F8686047
:103F4000B0BD00002DE9F04182B01E4690460D46FE
:103F50000446FEF749FC301A00EB0807FEF744FC64
:103F600040F21001C2F200010968C1F3CB3179437C
:103F7000019121688A682A40AA4227D1064618F191
:103F800001001FD0FEF730FC801BB84222D20198FE
:103F900001990028A1F1010101912168896808BFF8
:103FA000074601EA0500A842ECD00FE088682840E7
:103FB000A8420BD188682840A84207D188682840C9
:103FC000A84203D188682840A842EFD0002002B060
:103FD000BDE8F081D4E900014268B1F5827F22F0AA
:103FE000E00242600AD1A168B1F5004F02D0B1F5FC
:103FF000806F03D1016821F040010160A16AB1F531
:10400000005F07D1016821F400510160016841F4AB
:1040100000510160012084F85100002084F8500014
:10402000032002B0BDE8F08170470000FEF7E2BB5C
:1040300070470000406A0021C185C184FFF710BAB3
:1040400081B090F84210222921D183680246B3F54D
:10405000805F09D152F8281F52F8183C002B63D01A
:1040600003685B680AE000BF52F8281F13B90369B0
:10407000002BF5D003685B6803F07F030B701168B9
:1040800001311160C18D01390A04C18502D001B02E
:10409000704700BF0168CA6822F02002CA60CA687F
:1040A00022F48072CA604A6922F001024A6120212A
:1040B00080F8421000214163026B012A3CD1016368
:1040C000016851E8031F026821F0100142E8031360
:1040D000DBB1016851E8031F026821F0100142E8DA
:1040E000031393B1016851E8031F026821F0100126
:1040F00042E803134BB1016851E8031F026821F045
:10410000100142E80313002BDAD101680A68D206D5
:1041100006D5002200920A68009249680091009931
:10412000818D01B0FFF79AB9026852686FF35F2280
:1041300021F8022B8162A5E701B0FFF7FBBC00006C
:1041400040F26050C2F20000FFF78CB9FEE70000B9
:10415000B0F858C0BCF1000F04BF00207047036DD9
:1041600001465A1C50F82300142B08BF01220A658F
:10417000ACF10102A1F8582070470000B0F85820B7
:10418000142A0CD0D0F854C0BCF1130318BF0CF1A2
:104190000103436540F82310511CA0F85810B2F1F8
:1041A000140018BF0120704796B0FEF731FB0024C1
:1041B0000120CDE91144CDE90F440C9010904FF44B
:1041C000E0104FF48031022515900CA80694CDE93B
:1041D0000444CDE90D14CDE91351FEF7C9FD28B112
:1041E000EFF3108072B600BFFEE700BF0F20CDE9ED
:1041F00007054FF48060CDE90A0407A8022109945D
:10420000FEF7AEFC20B1EFF3108072B6FEE700BF00
:10421000022003904FF40040059003A8FEF71AFC1B
:1042200020B1EFF3108072B6FEE700BFFFF7D0FCBD
:10423000FFF78EFCFFF74AFDFFF724FD0CA8FDF702
:104240007FFDFFF767FD40F2D04540F20008C2F263
:10425000000501264FF008091024CCF2481800BFD1
:10426000FFF74EFE28680D9FFCF70DF80246002070
:1042700020210423CDF800900196B84768680D9F6F
:10428000FCF701F80246002028210423CDF8009015
:104290000196B8470E9F0020002142460323CDE936
:1042A00000640296B8470E9F6A680020102103231D
:1042B000CDE900640296B84715988047D0E702E040
:1042C00008C8121F08C1002AFAD1704770470020A1
:1042D00001E001C1121F002AFBD17047000000005D
:1042E00000000000010203040607080900000000A6
:1042F0000102030401020000F010101010FF101062
:104300001010F000000000000F04040404FF040477
:1043100004040F0000004040405F55555575555549
:10432000555F404040000040200F09498979090944
:10433000090F2040000000FE02424ACA4A4ACA4A07
:104340004A4202FE000000FF40504C4340404F50A4
:10435000505C40FF00000000F888888888FF88884B
:104360008888F800000000001F080808087F888877
:1043700088889F80F00080828282828282E2A2927C
:104380008A8682808000000000000040807F00005C
:10439000000000000000101010FF109008888888AE
:1043A000FF88888808000444827F01808040432C75
:1043B0001028468180000010101010D030FF30D03F
:1043C000121C1010000010080402010000FF000081
:1043D00001020408100004040484E43C272424247B
:1043E00024E40404040004020100FF090909094946
:1043F000897F0000000000FE225A8600FE92929201
:104400009292FE00000000FF04080700FF40200316
:104410000C1422414000008040201806800007183C
:104420002040800000000100207028262120202448
:104430003860000101000010129292929292921242
:104440001202FE0000000000003F101010103F009C
:1044500040807F000000000000C08080808080805D
:1044600080FC84808080808080C0C00000000000CC
:1044700000FF7F404040404040FF404040404040BF
:1044800040FF7F000000000000000000000000006E
:10449000007F70000000000000000000000000002D
:1044A00000000000000000000000000000FCF80018
:1044B00000000000000000000000000000000000FC
:1044C0000000FFFE020202020202020202FFFF02DD
:1044D0000202020202020202FF03000000000000CA
:1044E00000001F1F040404040404040404FFFF0468
:1044F00004040404040404041F000000000000007D
:10450000000000000000000000000000007F3F00ED
:10451000000000000000000000000000000000009B
:10452000000000000000000000000000000000008B
:104530000000000000000000000000F8F8F0F0703B
:10454000200000000000000000000000000000004B
:10455000000000000000000000000000000000005B
:1045600000000000000080000000000000000000CB
:104570000000000000000000000000FFFFFFFF003F
:10458000000000000000000000000000000000002B
:10459000000080800000000000000000000000001B
:1045A00000000000000000FFFFFE060606060606EB
:1045B0000606060606060606060606FFFFFFFF06B7
:1045C000060606060606060606060606060606068B
:1045D00006FFFFFFFF0702000000000000000000D0
:1045E00000000000000000FFFFFF000000000000CE
:1045F0000000000000000000000000FFFFFFFF00BF
:1046000000000000000000000000000000000000AA
:1046100000FFFFFFFF00000000000000000000009E
:1046200000000000000000FFFFFF181818181818FD
:104630001818181818181818181818FFFFFFFF185E
:1046400018181818181818181818181818181818EA
:1046500018FFFFFFFF000000000000000000000046
:104660000000000000000201010000000000000046
:104670000000000000000000000000FFFFFFFF003E
:10468000000000000000000000000000000000002A
:104690000001010000000000000000000000000018
:1046A000000000000000000000000000000000000A
:1046B0000000000000000000000000FFFFFFFF00FE
:1046C00000000000000000000000000000000000EA
:1046D00000000000000000000000000000000000DA
:1046E00000000000000000000000000000000000CA
:1046F00000000000000000000000001F1F0F0F005E
:1047000000000000000000000000000000000000A9
:104710000000000000000000000000000000000099
:10472000000000000000002F00000000070007004C
:1047300000147F147F1400242A7F2A120062640868
:1047400013230036495522500000050300000000E5
:104750001C224100000041221C000014083E0814E5
:104760000008083E0808000000A0600000080808D3
:104770000808000060600000002010080402003EED
:104780005149453E0000427F400000426151494688
:10479000002141454B31001814127F100027454578
:1047A0004539003C4A49493000017109050300368A
:1047B0004949493600064949291E0000363600009D
:1047C00000005636000000081422410000141414A2
:1047D000141400004122140800020151090600329D
:1047E0004959513E007C1211127C007F49494936DB
:1047F000003E41414122007F4141221C007F494946
:104800004941007F09090901003E4149497A007F79
:104810000808087F0000417F4100002040413F011F
:10482000007F08142241007F40404040007F020C7E
:10483000027F007F0408107F003E4141413E007F1F
:1048400009090906003E4151215E007F09192946E8
:104850000046494949310001017F0101003F4040C4
:10486000403F001F2040201F003F4038403F006372
:104870001408146300070870080700615149454394
:1048800000007F41410000552A552A550000414152
:104890007F0000040201020400404040404000004C
:1048A00001020400002054545478007F48444438E6
:1048B00000384444442000384444487F003854546D
:1048C000541800087E0901020018A4A4A47C007FEB
:1048D000080404780000447D4000004080847D008E
:1048E000007F102844000000417F4000007C041835
:1048F0000478007C0804047800384444443800FC00
:10490000242424180018242418FC007C080404081B
:1049100000485454542000043F444020003C404090
:10492000207C001C2040201C003C4030403C0044C7
:1049300028102844001CA0A0A07C004464544C44CF
:1049400014141414141400000000000000000000EF
:1049500000000000FC000000000002000000000C4D
:10496000020C020000000000000090D0BCD0BC90FF
:104970000003000300001824FE448C000302070219
:1049800001001824D8B04C80000300010201C03897
:10499000E438E00001020201020208060000000003
:1049A000000000000000000000F804020000000108
:1049B0000204000204F800000004020100009060FC
:1049C000F86090000000010000002020FC20200082
:1049D00000000100000000000000000008060000C8
:1049E0000000202020202000000000000000000027
:1049F000000000000002000000000080601C0200B7
:104A0000040300000000F8040404F800010202029C
:104A100001000008FC0000000002030200001884EE
:104A20004424180003020202020008042424D800CF
:104A300001020202010040B088FC80000000000377
:104A400002003C242424C400010202020100F824D4
:104A5000242CC0000102020201000C04E41C04002A
:104A6000000003000000D8242424D8000102020220
:104A7000010038444444F800000302020100000031
:104A800010000000000002000000000020000000F4
:104A90000000060000000020508804020000000012
:104AA0000102909090909000000000000000000231
:104AB000048850200002010000001804C4241800DB
:104AC000000002000000F804E494F8000102020271
:104AD000020000E09CF0800002030000030204FCDE
:104AE0002424D800020302020100F80404040C008C
:104AF00001020202010004FC0404F80002030202A5
:104B0000010004FC24740C0002030202030004FCF4
:104B100024740C00020302000000F0080444CC409E
:104B200000010202010004FC2020FC04020300003A
:104B300003020404FC040400020203020200000455
:104B400004FC040406040403000004FC24D00C0448
:104B500002030200030204FC04000000020302023C
:104B60000203FC3CC03CFC0003000300030004FC07
:104B700030C4FC04020302000300F8040404F8003B
:104B800001020202010004FC2424180002030200B6
:104B90000000F8848404F80001020207050004FC08
:104BA00024649800020302000302182424448C00A9
:104BB0000302020201000C04FC040C0000020302C8
:104BC000000004FC0000FC04000102020100047C5F
:104BD00080E01C040000030000001CE03CE01C001E
:104BE000000300030000049C609C04000203000317
:104BF0000200041CE01C04000002030200000C84FC
:104C0000641C04000203020203000000FE02020012
:104C1000000007040400000E30C000000000000186
:104C20000200000202FE000000040407000000046D
:104C3000020400000000000000000000000000006E
:104C40000808080808080000020000000000000032
:104C500000000040A0A0C00000010202030204FC0A
:104C60002020C00000030202010000C020206000DC
:104C700000010202020000C02024FC000001020228
:104C8000030200C0A0A0C000000102020200002038
:104C9000F82424040002030202000040A0A06020C7
:104CA00000070A0A0A0404FC2020C00002030200D4
:104CB00003020020E40000000002030200000000E4
:104CC00020E4000008080807000004FC80E0202021
:104CD0000203020003020404FC00000002020302BB
:104CE0000200E020E020C00003000300030020E0F9
:104CF0002020C00002030200030200C02020C000E8
:104D000000010202010020E02020C000080F0A027A
:104D1000010000C02020E0000001020A0F0820E08E
:104D2000402020000203020000000060A0A020003C
:104D30000002020203000020F8200000000001022F
:104D4000020020E00020E00000010202030220E057
:104D5000208060200000030100006080E08060008F
:104D600000030003000020608060200002030003B5
:104D7000020020E0208060200808070100000020D9
:104D8000A0602000000203020200000020DE0200FA
:104D9000000000070400000000FF00000000000FFA
:104DA00000000002DE2000000004070000000201F5
:104DB00002040402000000000000000000000000E7
:104DC00000000000000000000000000000F80000EB
:104DD0000000000000333000000000100C06100C32
:104DE0000600000000000000000040C07840C078CD
:104DF0004000043F04043F040400007088FC0830B5
:104E00000000001820FF211E0000F008F000E0184C
:104E1000000000211C031E211E0000F00888700005
:104E200000001E2123241927211010160E00000057
:104E300000000000000000000000000000E0180476
:104E40000200000000071820400000020418E000E3
:104E500000000040201807000000404080F0804023
:104E600040000202010F01020200000000F00000F9
:104E700000000101011F010101000000000000000D
:104E8000000080B070000000000000000000000082
:104E9000000000010101010101010000000000000B
:104EA00000000030300000000000000000008060C2
:104EB0001804006018060100000000E01008081047
:104EC000E000000F102020100F00001010F800006C
:104ED00000000020203F2020000000700808088803
:104EE00070000030282422213000003008888848D3
:104EF00030000018202020110E000000C02010F803
:104F0000000000070424243F240000F808888808D3
:104F100008000019212020110E0000E010888818D8
:104F20000000000F112020110E0000380808C838BA
:104F300008000000003F000000000070880808889A
:104F40007000001C222121221C0000E01008081023
:104F5000E0000000312222110F00000000C0C0005C
:104F60000000000000303000000000000080000061
:104F70000000000080600000000000008040201061
:104F8000080000010204081020004040404040405A
:104F900040000404040404040400000810204080BD
:104FA00000000020100804020100007048080808F2
:104FB000F0000000003036010000C030C828E810C2
:104FC000E0000718272423140B000000C038E0007D
:104FD0000000203C23020227382008F888888870C7
:104FE0000000203F202020110E00C03008080808D3
:104FF0003800071820202010080008F808080810BA
:10500000E000203F202020100F0008F88888E808E2
:105010001000203F20202320180008F88888E80886
:105020001000203F200003000000C03008080838AE
:10503000000007182020221E020008F808000008BF
:10504000F808203F210101213F20000808F8080846
:1050500000000020203F2020000000000808F80881
:105060000800C08080807F00000008F888C02818F1
:105070000800203F20012638200008F80800000022
:105080000000203F20202020300008F8F800F8F829
:105090000800203F003F003F200008F830C0000813
:1050A000F808203F200007183F00E010080808100B
:1050B000E0000F10202020100F0008F80808080852
:1050C000F000203F210101010000E0100808081055
:1050D000E0000F18242438504F0008F8888888888A
:1050E0007000203F2000030C302000708808080862
:1050F00038000038202121221C00180808F8080870
:1051000018000000203F2000000008F808000008F8
:10511000F808001F202020201F000878880000C801
:105120003808000007380E010000F80800F80008F1
:10513000F800033C0700073C0300081868808068FB
:10514000180820302C03032C30200838C800C83839
:1051500008000000203F2000000010080808C838A0
:1051600008002038262120201800000000FE02023E
:1051700002000000007F40404000000C30C00000F2
:105180000000000000010638C00000020202FE001C
:105190000000004040407F000000000004020202C6
:1051A00004000000000000000000000000000000FB
:1051B00000008080808080808080000202040000E7
:1051C00000000000000000000000000080808080DF
:1051D00000000019242222223F2008F800808000CD
:1051E0000000003F112020110E0000000080808090
:1051F0000000000E11202020110000000080808897
:10520000F800000E112020103F20000080808080D8
:105210000000001F222222221300008080F08888D4
:1052200088180020203F202000000000808080801F
:105230008000006B94949493600008F80080808054
:105240000000203F210000203F20008098980000AF
:1052500000000020203F20200000000000809898DF
:10526000000000C08080807F000008F8000080807F
:105270008000203F24022D302000000808F80000A4
:1052800000000020203F202000008080808080805F
:105290008000203F20003F20003F808000808080F1
:1052A0000000203F210000203F20000080808080FF
:1052B0000000001F202020201F0080800080800030
:1052C000000080FFA12020110E00000000808080DF
:1052D0008000000E112020A0FF8080808000808050
:1052E000800020203F21200001000000808080807D
:1052F00080000033242424241900008080E0808072
:1053000000000000001F20200000808000000080BE
:105310008000001F202020103F208080800000801F
:10532000808000010E30080601008080008000802F
:1053300080800F300C030C300F00008080008080D4
:1053400080000020312E0E312000808080000080FF
:10535000808080818E7018060100008080808080AF
:1053600080000021302C2221300000000000807CD1
:10537000020200000000003F404000000000FF006B
:10538000000000000000FF0000000002027C80001E
:1053900000000040403F0000000000060101020242
:1053A00004040000000000000000000000000000F5
:1053B00000000000000000000000000000000000ED
:1053C00000000000000000000000000000000000DD
:1053D000000000F0F0F000000000000000000001FC
:1053E0007F010000000000000000001C1C1C0000E9
:1053F000000000008060301C8C60301C0C0000003D
:10540000000000000000000000000000000000009C
:10541000000000000000000000E00000000000E0CC
:1054200000000086E69F86868686E69F860000014D
:105430001F01010101011F010100000080C0602067
:10544000F820E0C00000000003070C18FF70E181A5
:1054500000000000070F10107F100F070000806091
:10546000206080000000E02000000F3020309F709E
:10547000DC371030C0000000100E030007181018B1
:1054800007000000C02020E0C0000000000080E015
:105490001F38E88703C43C040000070F1810100BE6
:1054A000070D1010080000808C4C38000000000030
:1054B00000000000000000000000000000000000EC
:1054C00000000000000000000000000000000000DC
:1054D00080E0300804000000000000FEFF01000032
:1054E0000000000000000000030F1820400000042E
:1054F0000830E0800000000000000000000001FF14
:10550000FE0000000000004020180F030000000013
:105510000000000000000000C00000000000004289
:1055200066663C18FF183C666642000000000000FA
:1055300003000000000000000000000080000000E8
:105540000000001010101010FF10101010100000BC
:105550000000000003000000000000000000000048
:10556000000000000000000000000000000000003B
:10557000000000808C4C380000000000000000009B
:1055800000000000000000000000001010101010CB
:1055900010101010100000000000000000000000BB
:1055A00000000000000000000000000000000000FB
:1055B0000000000000000000000000001C1C1C0097
:1055C0000000000000000000000000000000E038C3
:1055D0000C000000000080701C0300000000006050
:1055E000380E0100000000000000000080C06020B4
:1055F0002060C080000000FEFF010000000001FFED
:10560000FE000001070E181010180E070100000020
:10561000808080C0E000000000000000000000FF6B
:10562000FF000000000000001010101F1F101010DD
:1056300000000080402020202060C0800000000387
:105640000300804020381F070000001C1A1918189A
:105650001818181F00000080C020202060C08000A3
:105660000000000303001010182FE780000000075F
:105670000F10101010180F070000000000000000AD
:10568000C0E0F000000000C0B088868180FFFF808D
:105690008000000000000010101F1F10100000000C
:1056A000E060606060606060000000003F1008081B
:1056B0000818F0E0000000070B101010101C0F037A
:1056C0000000000080C040202020E0C0000000FC5E
:1056D000FF211008080818F0E0000001070C18105E
:1056E0001010080F03000000C0E06060606060E020
:1056F0006000000003000000E01807000000000048
:105700000000001F1F00000000000080C06020207B
:10571000202060C080000087EF2C1818303068CF40
:10572000830000070F0810101010180F070000006A
:10573000C0C020202020C0800000001F3F604040EB
:10574000402010FFFE0000000C1C101010080F037A
:105750000000000000000000000000000000000049
:105760000000000E0E0E0000000000000000001CF3
:105770001C1C0000000000000000000000000000F1
:10578000000000000000000C0C0000000000000001
:105790000000005838000000000000000000000079
:1057A000008040201000000010284482010000000A
:1057B00000000000000000000102040810000000CA
:1057C0000000000000000000000000848484848445
:1057D0008484848484000000000000000000000035
:1057E00000000000102040800000000000000000C9
:1057F000000000000182442810000000100804028C
:1058000001000000000000C020201010101030E047
:10581000C0000003030000F010080C0703000000A4
:1058200000001C1C1C0000000000000000C04060C4
:1058300020202040C00000FCFF01F00E03C1FE0349
:10584000807F0001070E08111110110904020000E9
:10585000000080E0E000000000000000807C434089
:10586000477FF880000010181F1000000000131F71
:105870001C1020E0E02020202060C080000000FFFD
:10588000FF10101010182FE78000101F1F101010AD
:105890001010180F0700000080C04020202020605A
:1058A000E00000FCFF01000000000000010000011A
:1058B000070E181010100804030020E0E02020203C
:1058C0002040C080000000FFFF000000000001FF3A
:1058D000FE00101F1F10101018080E07010020E016
:1058E000E020202020202060800000FFFF1010100A
:1058F000107C00000000101F1F1010101010101856
:10590000060020E0E020202020206060800000FFD2
:10591000FF101010107C00000100101F1F1000006D
:10592000000000000000000080C06020202040E057
:10593000000000FCFF0100004040C0C140400001E9
:10594000070E181010100F0F000020E0E0200000DC
:10595000000020E0E02000FFFF101010101010FFEA
:10596000FF00101F1F1000000000101F1F1000007C
:10597000202020E0E020202000000000000000FFA8
:10598000FF000000000000001010101F1F1010107A
:10599000000000000000202020E0E0202020000087
:1059A0000000000000FFFF0000000060E080808039
:1059B000C07F3F00000020E0E020000020A0602029
:1059C000200000FFFF30187CE3C000000000101F23
:1059D0001F10000001131F1C181020E0E020000021
:1059E00000000000000000FFFF00000000000000B9
:1059F0000000101F1F10101010101018060020E0DB
:105A0000E0E000000000E0E0E02000FF013FFEC019
:105A1000E01E01FFFF00101F1000031F0300101FF6
:105A20001F1020E0E0C0000000000020E02000FF88
:105A30000003071C78E08000FF00101F100000002A
:105A40000000030F1F00000080C060202060C080A5
:105A5000000000FEFF010000000000FFFE0000014A
:105A6000070E181010180C07010020E0E02020207D
:105A7000202060C0800000FFFF2020202020301F59
:105A80000F00101F1F1000000000000000000000A9
:105A900080C060202060C080000000FEFF01000088
:105AA000000000FFFE000001070E1111133C7C678F
:105AB000210020E0E0202020202060C0800000FFA6
:105AC000FF101030F0D0080F0700101F1F1000004B
:105AD00000030F1C10100080C060202020204040D8
:105AE000E00000070F0C1818303060E08100001F44
:105AF0000C0810101010180F07008060202020E004
:105B0000E020202060800100000000FFFF00000076
:105B1000000100000000101F1F100000000020E026
:105B2000E020000000000020E02000FFFF00000057
:105B300000000000FF0000070F18101010101008E0
:105B400007002060E0E02000000020E0602000006E
:105B5000077FF88000807C03000000000000071F22
:105B60001C070000000020E0E02000E0E020002012
:105B7000E0200007FFF8E01FFFFCE01F000000002E
:105B8000031F0300011F03000000002060E0A000CD
:105B90000020E0602000000000038F7CF8C60100B8
:105BA00000000010181E130001171F1810002060BD
:105BB000E0E02000000020E06020000001073EF847
:105BC000E0180700000000000010101F1F10100058
:105BD000000000806020202020A0E0E020000000E5
:105BE0000000C0F03E0F0300000000101C1F171043
:105BF0001010101806000000000000FC040404044B
:105C000004000000000000FF000000000000000091
:105C10000000007F404040404000000010E00000D5
:105C200000000000000000000000031C6080000075
:105C3000000000000000000000030C708000000065
:105C40000404040404FC0000000000000000000044
:105C500000FF00000000000040404040407F000086
:105C6000000000000010080C040C081000000000E8
:105C70000000000000000000000000000000000024
:105C80000000000000000000000000000000000014
:105C90000000000000000000000000000000808004
:105CA00080808080808080808080000000040408E4
:105CB00008000000000000000000000000000000DC
:105CC00000000000000000000000000000000000D4
:105CD00000000000000000000000000098D84464AC
:105CE0002424FCF80000000F1F18101010081F1FBC
:105CF00010180020E0F0000000000000000000008C
:105D0000FFFF180804040CF8F00000001F0F181023
:105D10001010180F03000000000000000000000039
:105D2000000000E0F8180404043C38000000000300
:105D30000F0C1010101008060000000000000000FA
:105D40000020E0F0000000E0F81C04040408FFFF5D
:105D5000000000030F18101010081F0F08000000AB
:105D6000000000000000000000000000E0F84844CF
:105D700044444C7870000000030F0C1810101008F9
:105D800004000000000080C0602020E0C00000048B
:105D90000404FFFF040404040000000010101F1F8F
:105DA00010101000000000000000000000000000C3
:105DB0000000000070F88C04048CF874040C00706F
:105DC00076CF8D8D8D89C87870000020E0F00000BE
:105DD0000000000000000000FFFF08040404FCF8BD
:105DE000000000101F1F100000101F1F10000000F7
:105DF000000000606000000000000000040404FCDB
:105E0000FC000000000000001010101F1F101010F8
:105E100000000000000000000060600000000000C2
:105E20000000040404FCFC0000000000C0C08080EE
:105E3000C07F3F0000000020E0F0000000000000F4
:105E400000000000FFFF80C0F41C040400000010EC
:105E50001F1F1100031F1C1010000000202020E055
:105E6000F000000000000000000000FFFF00000044
:105E7000000000001010101F1F1010100000000084
:105E80000000000000000000000004FCFC0804FC0E
:105E9000FC0804FCFC00101F1F10001F1F10001F37
:105EA0001F100000000000000000000000000004BF
:105EB000FCFC08080404FCF8000000101F1F100080
:105EC00000101F1F10000000000000000000000074
:105ED000000000E0F0180C04040C18F0E0000003CF
:105EE0000F0C101010100C0F030000000000000039
:105EF0000000000000000004FCFC080404040CF88E
:105F0000F0000080FFFF889010101C0F03000000BD
:105F10000000000000000000000000E0F81C040485
:105F20000408F8FC000000030F1810109088FFFF11
:105F300080000000000000000000000000000404D9
:105F400004FCFC100804040C0C001010101F1F109F
:105F50001010000000000000000000000000000021
:105F6000000000003078CCC48484840C1C00000045
:105F70001E1810101011190F06000000000000C0BC
:105F800000000000000000040404FFFF04040400FB
:105F90000000000000000F1F1010100C0000000097
:105FA000000000000000000000000004FCFE0000F3
:105FB0000004FCFE000000000F1F181010081F0F47
:105FC00008000000000000000000000000000004C5
:105FD0000C3CFCC40000C43C0C0400000000010F99
:105FE0001E0E010000000000000000000000000084
:105FF0000000043CFCC400E47CFC84807C040000C1
:10600000071F070000071F07000000000000000036
:106010000000000000000004041C7CE4C0341C04E8
:1060200004000010101C1601131F1C1810000000A3
:106030000000000000000000000000040C3CFCC454
:1060400000C43C0404000000C080C1370E01000001
:106050000000000000000000000000000000000040
:106060001C0404C4F47C1C0400000000101C1F1756
:10607000111010180E0000000000000000F80C04C1
:10608000000000000000001028EF000000000000E9
:1060900000000000003F6040000000000000000021
:1060A000FF0000000000000000000000FF000000F2
:1060B0000000000000000000FF00000000000000E1
:1060C000040CF80000000000000000000000EF28B1
:1060D000100000000000000040603F0000000000D1
:1060E00000000018060202040810202030080000FA
:1060F00000000000000000000000000000000000A0
:1061000000000000000002030405060708090A0B4E
:106110000C0D0E0F10100000386100080000002068
:1061200018000000BE42000850610008180000205E
:1061300098090000CE420008010000001000000095
:1061400018040020740400200024F4000000000063
:04000005080000ED02
:00000001FF
